:020000040000FA
:100000008316FF239000003081001B3085000030F4
:100010009F008312073099003030900085016D20D9
:100020000518142805151028313090008E018F0115
:10003000051E1F280C1C182800000C10342847200F
:100040002008A1003030A1022108A800003078204B
:100050000530542047202008A20030302202A200A0
:10006000A800013078203A2800307320A100013028
:100070007320A2002108A3002208A400051568200F
:10008000A30B3F2805116820A40B43283A28051E1E
:100090004728051E4928C0308E00FF308F00051A02
:1000A0004F280E08A0000800A90005156D200511B5
:1000B0006D20A90B552808006430A500A50B5E280B
:1000C0000800A6005C20A60B62280800003061280A
:1000D000203061280230A7006F280430A700662076
:1000E000A70B6F28080083169B001C141A0887288A
:1000F00083169B008312280883169A001C1555301E
:100100009D00AA309D009C149C1884281C11831209
:100110000000080043006C00690067006E006F007B
:10012000740061006E00740020002D002000530058
:100130002E0020004C006900630068007400650018
:100140006E006200650072006700650072002000AA
:100150002D002000560065007200730069006F00DA
:100160006E002000310030002F00300034002F00DE
:040170003000380023
:0207FE002C3499
:02400E00D43F9D
:00000001FF
